:020000020000FC
:0200000012C02C
:0200140086C0A4
:02001A0050C0D4
:100026000FED0DBF08E101BB8A9A00E002BB00E0BC
:1000360003BF02E000BF07EC06BF01E009BF02E014
:1000460003BFD2D0F7D046D103E001B908E908B919
:100056004798789466276330F1F7ECD030E0442770
:10006600552766277727882704E0F0D0BB2730FD81
:1000760003D031FD0ED0FBCFE3D0082F06D10AE323
:1000860058D0072F02D10AE354D0062FFED03E7F68
:10009600089511E000E0E1D00B2FF7D000E249D03F
:1000A600E2EBF0E0E6D03D7F346008954576656E7C
:1000B6007428732920000F930FB7929A4395413005
:1000C60001F4423001F4423329F5442753955A305E
:1000D60009F49498A03011F0AA950AC032FD08C020
:1000E60008B1007221F0B3953260939A01C09398DB
:1000F600543679F45527949A316063956C3349F4F4
:10010600662773957C3329F477278395883109F41C
:100116008827000092980FBF0F9118950F930FB77D
:100126000F931F93A6E93B7F1F910F910FBF0F916E
:1001360018950F931F932F932FB72F93102F007F90
:10014600969A28B32F70022B08BB27D01295107FE2
:10015600969A122B18BB21D026D02F912FBF2F9104
:100166001F910F9108950F931F932F932FB72F93DE
:100176009698102F007F28B32F70022B08BB0DD046
:1001860096981295107F122B18BB07D00CD02F9182
:100196002FBF2F911F910F910895959A000000008F
:1001A6000000959808950F930FB70F9300E5000090
:1001B60000000A95E1F70F910FBF0F9108950F9375
:1001C6000FB70F931F9302E405C00F930FB70F935A
:1001D6001F9306E119EC1A95F1F70A95D9F71F91C5
:1001E6000F910FBF0F9108950F931F931FB72F9372
:1001F60007B3006F07BB8E9A8D9A26E0969895985E
:10020600DEDF2A95E9F703E008BBC7DFD8DFC5DFE5
:10021600D6DFC3DFD4DF02E008BBBFDFD0DF0CE2EE
:10022600A2DF0FE0A0DF04E09EDF2F911FBF1F912A
:100236000F9108950F9301E096DFC7DF0F910895A0
:100246000F9302E090DFC1DF0F9108950F930770BF
:10025600086089DFA8DF0F9108950F931F930F7130
:10026600117010FD10E4012B00687DDF1F910F91C6
:1002760008950F930FB70F930591003011F059DFD2
:10028600FBCF0F910FBF0F9108950F931F932F93DD
:100296002FB72F931CE9E12F10E0F12F00C0102F8C
:1002A60000E3145610F00395FCCF202F003309F01D
:1002B60009951C5900E31A5010F00395FCCF0995D7
:1002C600165F00E3010F09952F912FBF2F911F9104
:1002D6000F91089508E42DDF01E42BDF0CE429DFFC
:1002E6000CE427DF0FE425DF0AE223DF0AE221DF41
:0602F6000AE21FDF08957B
:00000001FF
